:100000000C9446000C9465000C9465000C946500FB
:100010000C9465000C9465000C9465000C946500CC
:100020000C9465000C946E000C9465000C946500B3
:100030000C9465000C9465000C9465000C946500AC
:100040000C9465000C9465000C9465000C9465009C
:100050000C9465000C9465000C9465000C9465008C
:100060000C9465000C9465000C9465000C9465007C
:100070000C9465000C9465000C9465000C9465006C
:100080000C9465000C943A050C94650011241FBE75
:10009000CFEFD0E1DEBFCDBF11E0A0E0B1E0E4E5FD
:1000A000FFE000E00BBF02C007900D92A030B10747
:1000B000D9F712E0A0E0B1E001C01D92A531B1076F
:1000C000E1F70E9498000C94A6070C9400008BE0C6
:1000D00085BD89EF83BD80E887BF08951F920F9289
:1000E0000FB60F9211248F939F93AF93BF9380917C
:1000F000000190910101A0910201B09103010196CC
:10010000A11DB11D8093000190930101A0930201F4
:10011000B0930301BF91AF919F918F910F900FBE4C
:100120000F901F90189585B390E3892785BB08959C
:10013000EF92FF920F931F938FEF84BBAC9AF894CA
:1001400089E08093140260E070E080E090E00E941B
:1001500017050E9405050E94670060E070E080E0DE
:1001600090E00E945D01EE24FF2409E010E021E010
:1001700030E040E050E060E070E08AE392E00E940E
:10018000F30278940E94EB03FDCFEF92FF920F935E
:100190001F93DF93CF9300D000D0CDB7DEB78C0193
:1001A000FC0183899489029709F07CC08281853A99
:1001B00009F05EC08581E82FF0E0EE0FFF1FEC5FD5
:1001C000FE4F8081918101969183808385B390E376
:1001D000892785BBF8018581A581E82FF0E0EE0F26
:1001E000FF1FEC5FFE4FB0E0AA0FBB1FA85FBE4F22
:1001F000208131818D919C912817390709F052C0D7
:1002000089E08983F8018581882369F460E070E0E2
:1002100080E090E00E947C0185E08A839091040157
:10022000809105010CC060E070E080E090E00E94E9
:10023000800186E08A8390910601809107018B837B
:100240009C8344E0BE016F5F7F4F81E00E944B07BB
:1002500092E3E92EF12C01E010E020E030E040E0F4
:1002600050E060E070E084E891E00E94F3021AC080
:10027000F801828160E070E090E00E941A02F801CB
:10028000828123813481881F8827881FE82FF0E02E
:10029000EE0FFF1FE85FFE4F922F80E0830F911D4E
:1002A000918380830F900F900F900F90CF91DF91EB
:1002B0001F910F91FF90EF90089584B3836084BBEA
:1002C00085B38C7F85BB84B38C6084BB85B3837F0F
:1002D00085BB1ABA8FEF8BBB81E080930C01089528
:1002E000A998A89A0895A898A99A0895AB98AA9A47
:1002F0000895AA98AB9A089585B38C7F85BB08951D
:1003000085B3837F85BB0895892B09F064C0E1998B
:10031000FECF1FBA1EBAE09A3DB3E199FECF81E04D
:1003200090E09FBB8EBBE09A2DB3932F80E040916D
:10033000040150910501420F511D480F591F1092A1
:10034000050110920401E199FECF1FBA1EBA5DBBF0
:100350000FB6F894E29AE19A0FBEE199FECF81E0E0
:1003600090E09FBB8EBB4DBB0FB6F894E29AE19A2A
:100370000FBEE199FECF82E090E09FBB8EBBE09A7A
:100380003DB3E199FECF83E090E09FBB8EBBE09A46
:100390002DB3932F80E04091060150910701420F49
:1003A000511D480F591F1092070110920601E19943
:1003B000FECF82E090E09FBB8EBB5DBB0FB6F89492
:1003C000E29AE19A0FBEE199FECF83E090E09FBBF5
:1003D0008EBB4DBB29C0E199FECF1FBA1EBA1DBA14
:1003E0000FB6F894E29AE19A0FBEE199FECF81E050
:1003F00090E09FBB8EBB1DBA0FB6F894E29AE19ACB
:100400000FBEE199FECF82E090E09FBB8EBB1DBA8C
:100410000FB6F894E29AE19A0FBEE199FECF83E01D
:1004200090E09FBB8EBB1DBA0FB6F894E29AE19A9A
:100430000FBE08959C018270907027FF0DC0892B1C
:1004400041F020FF03C0AB98AA9A0895AA98AB9AEE
:10045000089585B3837F0CC0892B41F020FF03C032
:10046000A998A89A0895A898A99A089585B38C7F09
:1004700085BB0895EF92FF920F931F93DF93CF9365
:1004800000D000D0CDB7DEB7C9990EC0A898909122
:1004900004012091050180910C01882309F450C0CA
:1004A0009C832B8381E02DC0C8990EC0A9989091A0
:1004B00004012091050180910C01882309F440C0BA
:1004C0009C832B8382E01DC0CB990DC0AA9890918C
:1004D00006012091070180910C01882389F19C83FA
:1004E0002B8383E00EC0CA9928C0AB989091060177
:1004F0002091070180910C01882311F19C832B83AB
:1005000084E08A8389E0898344E0BE016F5F7F4F86
:1005100081E00E944B0710920C0182E3E82EF12C3F
:1005200001E010E020E030E040E050E061E070E009
:1005300084E891E00E94F30203C081E080930C0103
:100540000F900F900F900F90CF91DF911F910F910F
:10055000FF90EF90089587B3806C87BBC09A88E2C4
:100560008FBD82E18EBD80E29EE497BD86BD8CED9D
:1005700095E099BD88BD90937900809378000895A7
:10058000672B19F499BD88BD0895909379008093E5
:1005900078000895089588B599B5895E934050F420
:1005A0001AC088B599B5019799BD88BDC901019751
:1005B000F1F702C020E137E288B599B5885E934033
:1005C00081F7089588B599B5019699BD88BDC9018F
:1005D0000197F1F702C020E137E288B599B580565E
:1005E000994081F70895CF92DF92EF92FF920F9397
:1005F0001F93CF93DF93EC016B01A0E0B0E09A2F43
:10060000FD0184E0EE0FFF1F8A95E1F7EA0FFB1F63
:10061000E35FFE4F8785882329F09F5F1196AC30FA
:10062000B10569F7692F70E0FB01A4E0EE0FFF1F31
:10063000AA95E1F7E60FF71FE35FFE4FD183C08372
:10064000D382C2825583448337832683E114F10425
:1006500011F4108A08C082E3E816F10411F481E075
:1006600001C082E0808BFB0134E0EE0FFF1F3A9562
:10067000E1F7E60FF71FE35FFE4FA089B0E0A75256
:10068000BE4F8C91982F9E0D96878F5F8C9311870C
:10069000008781E08787F894209100013091010163
:1006A0004091020150910301C801A0E0B0E0820F27
:1006B000931FA41FB51FFB0124E0EE0FFF1F2A9517
:1006C000E1F7E60FF71FE35FFE4F82879387A4876A
:1006D000B5877894DF91CF911F910F91FF90EF90A4
:1006E000DF90CF900895CF92DF92EF92FF920F9319
:1006F0001F93CF93DF93DC01EB01690120E030E031
:10070000622FF90174E0EE0FFF1F7A95E1F7E20F17
:10071000F31FE35FFE4F8785882331F06F5F2F5F04
:100720003F4F2C30310561F7262F30E0F90164E0AE
:10073000EE0FFF1F6A95E1F7E20FF31FE35FFE4F35
:10074000B183A083D383C28355834483D782C68277
:10075000E114F10411F4108A08C082E3E816F104F0
:1007600011F481E001C082E0808BB90194E0660F52
:10077000771F9A95E1F7620F731F635F7E4FEB015E
:10078000E889F0E0E752FE4F8081982F9E0D9E870A
:100790008F5F80831987088781E08F872091000110
:1007A000309101014091020150910301C801A0E084
:1007B000B0E0820F931FA41FB51FFB0182879387B0
:1007C000A487B587DF91CF911F910F91FF90EF9094
:1007D000DF90CF900895EF92FF920F931F93CF93E6
:1007E000DF93F894E0900001F09001010091020184
:1007F0001091030178941092DC018091DF018F5FEA
:100800008093DF018091DF01883C49F48091DE0113
:1008100086958093DD011092DE011092DF014FEF8B
:100820005FEF20E030E0F901A4E0EE0FFF1FAA9592
:10083000E1F7E20FF31FE35FFE4F8785882399F00E
:100840008091DC018F5F8093DC0182859385A48594
:10085000B585E816F9060A071B0728F0868585176F
:1008600010F45685422F2F5F3F4F2C303105D9F6BB
:100870004F3FB9F18091DE018F5F8093DE01842FBD
:10088000992787FD9095EC01E4E0CC0FDD1FEA95F8
:10089000E1F7C80FD91FC35FDE4FE881F9816C8192
:1008A0007D818A819B8109958E819F81892B49F465
:1008B0001F86E889F0E0E752FE4F808181508083F7
:1008C00010C02A853B854C855D8588859985A0E08B
:1008D000B0E0820F931FA41FB51F8A879B87AC8748
:1008E000BD8781E0DF91CF911F910F91FF90EF9035
:1008F00008959C01DB0160E070E0FB0144E0EE0F35
:10090000FF1F4A95E1F7E60FF71FE35FFE4F808177
:1009100091818217930719F58785882301F1F8944F
:100920002091000130910101409102015091030199
:10093000CD01A0E0B0E0820F931FA41FB51FFB0103
:1009400024E0EE0FFF1F2A95E1F7E60FF71FE35FA4
:10095000FE4F82879387A487B587789408956F5F49
:100960007F4F6C30710549F60895AC0120E030E00E
:10097000F901A4E0EE0FFF1FAA95E1F7E20FF31FC4
:10098000E35FFE4F8081918184179507B9F48785D5
:100990008823A1F0209100013091010140910201D2
:1009A00050910301CB01A0E0B0E0820F931FA41F80
:1009B000B51F82879387A487B58708952F5F3F4F20
:1009C0002C303105A9F60895AC0120E030E0F901A2
:1009D000B4E0EE0FFF1FBA95E1F7E20FF31FE35FFC
:1009E000FE4F808191818417950749F41786E0892D
:1009F000F0E0E752FE4F80818150808308952F5FA1
:100A00003F4F2C30310519F7089580E090E0FC014C
:100A100024E0EE0FFF1F2A95E1F7E80FF91FE35FCF
:100A2000FE4F178601968C30910589F708958091C5
:100A30001402880F81608093720080E480937000BC
:100A4000E1E7F0E080818C7F80832FEF20937300BB
:100A500085EC8093740081E090E09093E3018093B3
:100A6000E2011092E10120930E021092F80110921F
:100A7000F70108951F920F920FB60F920BB60F92C7
:100A80001124EF92FF920F931F932F933F934F9355
:100A90005F936F937F938F939F93AF93BF93EF93E6
:100AA000FF938091E2019091E301817C09F4CBC036
:100AB0008091710090E0887F90708038910561F19D
:100AC00081389105ACF48836910509F48AC08936DD
:100AD00091052CF48036910509F0B3C09AC0803797
:100AE000910509F496C08837910509F0AAC079C02C
:100AF0008039910589F0813991052CF48838910568
:100B000009F09FC096C08839910509F492C0803AD7
:100B1000910509F096C093C08091E2019091E301A4
:100B20008034910581F4809173008093E5018FEF0B
:100B300080930E0280E890E09093E3018093E201BD
:100B40001092E1017CC08091E2019091E301803834
:100B5000910509F074C09091E1018091E501981729
:100B6000A0F48091E101E82FF0E090917300EC5146
:100B7000FE4F92838F5F8093E10190910E028091EE
:100B80007300892780930E025AC08091E101803161
:100B900011F5809173008093F60190910E0280917F
:100BA000F601981719F081E090E002C082E090E031
:100BB0009093F8018093F701EE24FF2400E010E009
:100BC00020E030E040E050E064EE71E085EC90E041
:100BD0000E9473032EC08091E1018F5F8093E10139
:100BE0002EC0809112028F5F8093120280910F02BB
:100BF0008A3078F422E3E22EF12C02E310E020E0C8
:100C000030E040E050E060E070E08FE097E00E946C
:100C10007303809173008093E4011092F8011092A5
:100C2000F7011092E10185EC8093740080E490E07C
:100C30007DC081E090E09093E3018093E20185EC38
:100C4000D5C085E4D3C08091710090E0887F90701A
:100C50008032910509F49CC08132910554F48031B1
:100C6000910599F088319105D1F0089709F0B7C046
:100C70000CC08033910509F45EC08833910509F4F6
:100C800060C0889709F0ABC011C08091F9018093D2
:100C9000730085E88093740088E090E047C010926C
:100CA000E0018091FA01809373003BC08091E001E4
:100CB0008131D9F485E98093740080E290E09093CB
:100CC000E3018093E20110920F0280911002909153
:100CD00011020196909311028093100260E070E07F
:100CE00087E195E00E94B50483C09091E001809176
:100CF000FA01981750F080910B0280937300809155
:100D0000E0018F5F8093E0010CC09091E001E92F3A
:100D1000F0E0E750FE4F8281809373009F5F9093D5
:100D2000E00185E88093740080E190E09093E30116
:100D30008093E2015DC0809112028F5F8093120266
:100D40002CC0809112028F5F8093120260E070E0ED
:100D500087E195E00E94B50480910F028A3080F40B
:100D600092E3E92EF12C02E310E020E030E040E0D5
:100D700050E060E070E08FE097E00E94730306C0EF
:100D800088E290E09093E3018093E20185E82EC031
:100D9000809113028F5F8093130260E070E087E11F
:100DA00095E00E94B50480910F028A3080F482E3BE
:100DB000E82EF12C02E310E020E030E040E050E0CB
:100DC00060E070E08FE097E00E94730306C088E265
:100DD00090E09093E3018093E20185E907C084E00D
:100DE00090E09093E3018093E20185E080937400AA
:100DF000FF91EF91BF91AF919F918F917F916F91F3
:100E00005F914F913F912F911F910F91FF90EF9024
:100E10000F900BBE0F900FBE0F901F901895EF9282
:100E2000FF920F931F938091E2019091E30101974C
:100E300071F042E3E42EF12C05E010E020E030E018
:100E400040E050E060E070E08FE097E01DC010925D
:100E5000E00185EA8093740082E090E09093E301E2
:100E60008093E20180910F028F5F80930F0232E343
:100E7000E32EF12C00E117E220E030E040E050E00A
:100E800060E070E087E195E00E94F3021F910F910E
:100E9000FF90EF900895EF92FF920F931F93582FBA
:100EA00080910F02882309F448C080910F028A3094
:100EB00009F443C081E03CC08FEF80930B02DB015B
:100EC00020E030E00DC08C91F901E750FE4F8283A5
:100ED00080910B029D91892780930B022F5F3F4FDA
:100EE000241788F381E080930F02852F90E0880F0C
:100EF000991F8093F9014093FA011092E00185EA6D
:100F00008093740082E090E09093E3018093E2018B
:100F100052E3E52EF12C05E010E020E030E040E067
:100F200050E060E070E087E195E00E94F30280E02D
:100F30001F910F91FF90EF9008958091E2019091A1
:100F4000E301019709F4B8CF82E0F2CFF89400C032
:040F5000F894FFCF43
:00000001FF
